:1000000020C190C239C138C137C1C9C835C134C156
:10001000F6C832C131C130C12FC12EC12DC12CC192
:100020002BC12AC129C1040309041803720061000D
:10003000700068006E00650074002E006E006500A0
:1000400074000A0331003000300030000501150053
:1000500026FF0075080904A1010901A10009300962
:100060003195028182C0A100093209339502818253
:10007000C0093409350936093795048182C0050164
:100080000902A1010901A1000509190129021500B0
:10009000250195027501810295017506810305010F
:1000A000093009311581257F750895028106C0C088
:1000B00012010101000000088117971A07020102CE
:1000C000030105010905A1010901A1000930093158
:1000D000150026FF00750895028102C00509190167
:1000E0002904150025017501950481027501950407
:1000F0008103C012010101000000088117990A075D
:1001000002010000010501150026FF007508090421
:10011000A1010901A1000930093195028182C0A124
:10012000000932093395028182C009340935093644
:10013000093795048182C012010101000000088185
:1001400017961A0702010203010501150026FF0098
:1001500075080904A1010901A100093009319502BE
:100160008182C0A1000932093395028182C009341D
:1001700009350936093795048182C005010904A1B2
:10018000010901A100850109300931150026FF0090
:100190007508950281020509190129081500250134
:1001A000750195088102C0C005010904A10109017A
:1001B000A100850209300931150026FF0075089558
:1001C000028102050919012908150025017501950B
:1001D000088102C0C005010904A1010901A100852F
:1001E0000309300931150026FF00750895028102C8
:1001F00005091901290815002501750195088102D5
:10020000C0C005010904A1010901A100850409304C
:100210000931150026FF00750895028102050919AC
:1002200001290815002501750195088102C0C01239
:100230000101010000000881179D0A070201020365
:10024000010011241FBECFE5D4E0DEBFCDBF11E019
:10025000A0E6B0E0EAE0F7E102C005900D92A23519
:10026000B107D9F711E0A2E5B1E001C01D92AC3FA2
:10027000B107E1F737D347CAC3CE85B7836085BFDF
:100280008BB780648BBF83EC8093C20108950F937A
:100290001F93CF93DF939091D20119160CF0A6C053
:1002A0002091CF018091CE018D3209F095C08AE571
:1002B000809361009B3009F08FC0CCE0D0E0C21B7E
:1002C000D109CA52DE4F8881807609F077C010923A
:1002D000C0018981882351F41092C10180EC91E022
:1002E0009093D1018093D00132E06BC0853021F42E
:1002F0008A818093D30160C0863009F043C08B812E
:100300008130E1F1823019F4CE016FD259C08330CF
:1003100049F58A81882341F486E290E09093D101E7
:100320008093D00134E050C0813041F48AE290E003
:100330009093D1018093D00138E146C0823041F4DE
:1003400083E690E09093D1018093D00136E339C0E9
:100350008330C9F582E490E09093D1018093D0017D
:100360003CE032C0813241F485E691E09093D101C6
:100370008093D00139E028C0823229F5CE0135D2F0
:10038000382F22C0883019F485ED91E00AC08930F9
:1003900021F48A818093D5010FC08A3041F480EC2A
:1003A00091E09093D1018093D00131E00AC08B306D
:1003B00019F483EC8093C20130E003C0CE0143D234
:1003C000382F20E802C030E020EC8F81882339F4F8
:1003D0008E81831728F003C080E020E801C0832FBE
:1003E00020935201809360001092D20180916100AD
:1003F00084FF49C0809160008F3F09F444C0182FEA
:10040000893008F018E0811B8093600080915201D0
:1004100080FD02C00BE401C003EC8F5F80935201AA
:100420002091D0013091D10186FD05C0D901912FD5
:10043000E8EBF1E011C0A8EBB1E080E090E006C08D
:10044000F901E80FF91FE491ED9301961817C1F730
:1004500005C08D91819391509923D9F7F901E10F4E
:10046000F11DF093D101E093D00188EB91E0612F71
:1004700055D0183019F08FEF809360000093B701CA
:100480001C5F109361009AE080B3847131F4915045
:10049000D9F71092D3011092CD01DF91CF911F9126
:1004A0000F9108951F93DC01162F8091620084FF45
:1004B0000AC08091C20198E889278093C201912FD8
:1004C000E3ECF1E007C08AE580936200F8CF8D91FC
:1004D000819391509923D9F783EC91E0612F1ED03D
:1004E0001C5F109362001F910895A82FB92F8FEF02
:1004F0009FEF41E050EA615070F02D9138E0722F8B
:10050000782796958795269570FF02C084279527B2
:100510003A95A9F7F0CF809590950895E6DF8D93F1
:100520009D930895CF93CFB7CF93849BFECF849BA9
:1005300009C0849B07C0849B05C0849B03C0849B27
:1005400001C09EC0DF93C091CF01DD27CA52DE4FAC
:10055000849B02C0DF91EBCF2F930F931F9300B3C7
:100560002FEF04FB20F94F933F9310B34FEF012778
:1005700004FB21F93BE031C04E7F012F10B3216015
:1005800028C0102F4D7F2260000000B329C04B7F90
:100590002460012F000010B32BC010B3477F2860E8
:1005A0002AC04F7E00B320612CC04F7D10B3206263
:1005B0002FC04F7B00B3206432C0422700B3499361
:1005C0004FEF0000102714FB20F910B31471A9F1AC
:1005D000297F91F2012704FB21F900B3237F89F2DF
:1005E0003150F0F1102714FB22F910B3277E79F275
:1005F000012704FB23F92F7C81F200B3102714FBA1
:1006000024F92F7971F200C010B3012704FB25F9FA
:100610002F7359F200C000B3102714FB26F92230C3
:1006200040F200C010B3012704FB27F9243028F65C
:100630004F77206810B30000F9CF3B50319533302D
:1006400010E41ABFB8F0C31BD0400881033C41F14D
:100650000B3431F11981412F1F772091CD011217F1
:1006600031F4093691F10D3279F0013E69F022271B
:100670002093D4013F914F911F910F912F91DF91C2
:10068000CF91CFBFCF9118950093D4013F914F9157
:100690001F910F912F91DF91CAB7C6FD46CFF0CFC2
:1006A0000091D401002331F31091D2011123A1F55F
:1006B0003430A2F13093D2010093CE011091CF01DA
:1006C0003BE0311B3093CF0129C00091D2010130B2
:1006D0001CF50AE547FD09C03091610034FD20C0DA
:1006E00000936100C7EBD1E01FC03091620034FD80
:1006F00017C000936200C2ECD1E016C0052710E0DD
:1007000002BB1FC0052722C0052727C005272CC014
:10071000052710E002BB33C04AE503C042ED01C02B
:10072000432FC4E1D0E032E011B31461949A02B3D4
:1007300011BB5F9354E120E820FF052702BB2795FA
:1007400017951C3FD8F620FF0527279502BB179564
:100750001C3FC0F620FF05272795179502BB1C3FBD
:1007600098F620FF0527279517951C3F02BB70F6CA
:1007700000C0499120FF052702BB279517951C3F14
:1007800038F620FF0527279502BB17951C3F38F543
:1007900020FF05272795179502BB1C3F10F520FF6A
:1007A0000527279517951C3F02BBE8F4242F3A959F
:1007B00019F60B7E5F9102BB00C01091D301C651A8
:1007C000D04011F01093CD0110E41ABF006111B3B5
:1007D0001B7E402F4B7E02BB11BB42BB4BCF05277C
:1007E000D3CF0527D8CF0527DDCFFC0180818076C8
:1007F00041F58181863029F583818230D1F08232C2
:1008000069F08130F1F480915701909158019093F3
:10081000D1018093D00180915901089580915401B4
:10082000909155019093D1018093D0018091560110
:10083000089587E990E09093D1018093D00182E2FE
:10084000089580E00895DC012AE631E03093D1017B
:100850002093D0018C918076803209F041C01196AE
:100860008C911197823081F08A30F1F08130C1F59E
:10087000E0915A01F0915B010088F189E02DC901F6
:1008800012966C910995089512969C91892F81502A
:10089000883030F5892F90E08F599E4F9093D10189
:1008A0008093D00181E008951296EC911297EE2387
:1008B00059F4E2E6F1E013968C911397819381E06D
:1008C000EA36F807C1F70CC08E2F8150883040F40B
:1008D000F0E0EF59FE4F13968C91808380E00895ED
:1008E00080E008958F929F92AF92BF92CF92DF9255
:1008F000EF92FF920F931F93DF93CF93CDB7DEB7A5
:10090000AA970FB6F894DEBF0FBECDBF88E0FE01F8
:100910003196DF01982F1D929A95E9F7E2E6F1E012
:10092000DF011D928A95E9F787B3897F87BB88B37A
:10093000866088BB80E395E70197F1F7AFD4FC01AF
:1009400090935B0180935A010284F385E02D099511
:100950008823B9F0DE011996E9EBF0E082E201901C
:100960000D928150E1F7A3E6B0E0FE01399682E2F4
:1009700001900D928150E1F725D690935B01809311
:100980005A01E0915A01F0915B0184819581909325
:100990005501809354018281809356018085918511
:1009A000009731F09093580180935701868107C0DA
:1009B00087E391E09093580180935701A1D48093ED
:1009C0005901809156018093B00014BA8FEF85BB16
:1009D00088EF82BB85E081BB11BA83BF8FE085BD04
:1009E00084EC83BDE0915A01F0915B010284F385B0
:1009F000E02D099542DC789411E0882483945E010F
:100A00000894A11CB11C91E0C92ED12C80E8982E2D
:100A100001C010E0A8953BDC112341F0E0915A01A0
:100A2000F0915B010484F585E02D099508B600FC82
:100A300002C0FF2428C088BE40915A0150915B013A
:100A4000D501FF2420E030E018C0F901EE59FE4F37
:100A5000E081EE2379F08C91853018F085508C93ED
:100A600009C0EC93C601022E02C0880F991F0A9498
:100A7000E2F7F82A2F5F3F4F1196FA0180819181AA
:100A80002817390714F308B607FE27C098BEE0916F
:100A90005A01F0915B010484F585E02D099500E091
:100AA00010E012C00684F785E02D802F8F5F099536
:100AB000882341F0C601002E02C0880F991F0A94B6
:100AC000E2F7F82A0F5F1F4FE0915A01F0915B01A6
:100AD00080819181081719072CF3FF2009F499CF21
:100AE000A39AAB9800E010E0EF2CFF24E7FCF09411
:100AF00022C0C701002E02C0959587950A94E2F79F
:100B000080FF17C08091620084FF13C0602F6F5F69
:100B10000088F189E02D8CE591E00995682F8CE53E
:100B200091E0C0DC02C0B3DBA8958091620084FF35
:100B3000FACF0F5F1F4FE0915A01F0915B01808166
:100B4000918108171907ACF2AB9A63CFAC9A80E396
:100B50008A95F1F7AC9880E090E030E048E1242FEE
:100B60002A95F1F7AD98330F9B9B3160242F2A957E
:100B7000F1F7AD9A01968830910589F730937101AC
:100B800080E090E048E1242F2A95F1F7AD98369562
:100B90009B9B3068242F2A95F1F7AD9A01968830F7
:100BA000910589F73093720108951F931FB7F89448
:100BB000A49AA59AA398AB9AAD9AAC98C7DF1FBF29
:100BC00080E01F9108958CE490E09093E000809382
:100BD000DF008BED90E00895FC01009709F453C00D
:100BE000A091710180917201682F70E0CB01807F2C
:100BF0009070803F910521F481E08093700102C0E4
:100C0000109270014A2F50E0A0FD03C020E830E0B0
:100C100002C02FEF30E041FF02C020E030E042FD93
:100C200003C080E890E002C08FEF90E043FF02C075
:100C300080E090E020838183CA018074907025E079
:100C4000959587952A95E1F79A0120723070B3E067
:100C500035952795BA95E1F7982F922BAA1FAA27C9
:100C6000AA1F9A2B4071507055954795942B9283EB
:100C700080917001882339F484E0660F771F8A958C
:100C8000E1F7962B9283809171019091720190937C
:100C900074018093730183E008958091ED00909139
:100CA000EE00892B31F01092EE001092ED0081E001
:100CB000089581E791E063E771E042E050E002D5FA
:100CC0000895FC01AC9A80E38A95F1F7AC9890E026
:100CD00028E1822F8A95F1F7AD98822F8A95F1F756
:100CE000AD9A9F5F9830A9F7908120E038E1832F7B
:100CF0008A95F1F7AD98990F9B9B9160832F8A9508
:100D0000F1F7AD9A2F5F283091F790830895DF9324
:100D1000CF930F92CDB7DEB7CE010196D2DF90E030
:100D200089818F70813009F491E0892F0F90CF91E4
:100D3000DF9108956F927F928F929F92AF92BF92B0
:100D4000CF92DF92EF92FF920F931F93DF93CF9397
:100D50000F92CDB7DEB773E0E72EF12CE822F9222F
:100D600006E010E04E010894811C911C68EBA62E51
:100D70006BE0B62E54E0752E40E3642E30E8C32EAF
:100D80003BEBD32EC4019DDF898190E0807390708E
:100D900024E0959587952A95E1F78E159F0529F40E
:100DA000F0927E01E0927D011CC0C5010197F1F730
:100DB00080E090E0AC9A272D2A95F1F7AD98AD9A96
:100DC000272D2A95F1F7AC98262D2A95F1F7019653
:100DD0008F31910579F7C6010197F1F70150104065
:100DE00089F60F90CF91DF911F910F91FF90EF90B7
:100DF000DF90CF90BF90AF909F908F907F906F903B
:100E00000895DF93CF930F92CDB7DEB7CE01019651
:100E100058DF2981822F8F70813079F580917B0195
:100E200090917C01892B71F522952695269523704A
:100E3000822F90E08130910571F0823091051CF491
:100E4000892B79F013C08230910541F0039771F43A
:100E500080E090E00AC081E090E007C082E090E08E
:100E600069DF80917D0190917E0164DFCE01019662
:100E700028DF89818F70813029F010927C011092D7
:100E80007B0156C081E090E090937C0180937B01D0
:100E9000898180937F0180E797E10197F1F78CEDDD
:100EA00095E00197F1F780E090E050E030E2232FE9
:100EB0002A95F1F7AD98550F9B9B51600000AD9AB4
:100EC00001968830910599F780E090E030E040E2AB
:100ED000242F2A95F1F7AD98330F9B9B31600000CA
:100EE000AD9A01968830910599F7232F2F77452FDA
:100EF0004F7737FD219557FD4195332727FD3095D5
:100F00008091750190917601820F931F90937601E5
:100F100080937501242F332727FD30958091770129
:100F200090917801820F931F9093780180937701BD
:100F30000F90CF91DF910895A49AA59AA398AB9AA8
:100F4000AD9AAC985EDF80917F01829586958695FB
:100F5000837090E08130910571F0823091051CF42E
:100F6000892B31F00EC08230910541F0039749F48E
:100F700080E090E005C081E090E002C082E090E077
:100F8000D9DE80E008958091010190910201892BC2
:100F900029F010920201109201011DC090917F0171
:100FA000809180019817B9F42091750130917601F4
:100FB00080918101909182012817390761F440E006
:100FC0002091770130917801809183019091840183
:100FD0002817390709F041E0842F0895FC01009794
:100FE00009F454C08091790190917A01892B41F0E4
:100FF00010821182128210927A011092790146C0F9
:10100000A0917F018A2F8295869586958370808333
:1010100060917501709176018FEF6138780714F453
:1010200081E806C06038710514F08FE701C0862F93
:1010300040917701509178019FEF4138590714F49E
:1010400021E806C04038510514F02FE701C0242FD5
:1010500081832283992787FD9095909382018093C5
:101060008101332727FD309530938401209383013C
:10107000A0938001681B790B7093760160937501D2
:10108000421B530B509378014093770183E00895FE
:101090008EE790E09093F4008093F30080EB90E073
:1010A0009093F8008093F7008FEE90E00895A49A53
:1010B000A59AA398AB9AAD9AAC9880E00895AC9AA3
:1010C00080E38A95F1F7AC9880E090E030E048E169
:1010D000242F2A95F1F7AD98330F9B9B3160242F75
:1010E0002A95F1F7AD9A01968830910589F73093EA
:1010F000850108958091850190918601891B08954D
:10110000FC010097B9F160918501462F50E060FD28
:1011100003C020E830E002C02FEF30E041FF02C002
:1011200020E030E042FD03C080E890E002C08FEF95
:1011300090E043FF02C080E090E0208381839A0129
:101140002074307075E0359527957A95E1F7CA01DE
:101150008072907033E0959587953A95E1F7282B4A
:10116000661F6627661F262B407150705595479560
:10117000242B2283809185018093860183E008954A
:1011800082EC90E0909308018093070183EF90E058
:1011900090930C0180930B0183E091E008951F92DE
:1011A0000F920FB60F9211242F933F938F93EF93CB
:1011B000FF932CB53DB51DBC1CBC8091150187FD6E
:1011C0000FC08091150186305CF4E0911501FF2776
:1011D000E7FDF095EE0FFF1FE451FE4F31832083B2
:1011E000809115018F5F80931501FF91EF918F9191
:1011F0003F912F910F900FBE0F901F9018951F9247
:101200000F920FB60F9211248F938FEF80931501D9
:101210008F910F900FBE0F901F901895E82FF0E060
:10122000EE0FFF1FE451FE4F808191812EE2803E40
:10123000920710F480EE9EE2805E9E426DE270E0C6
:101240004ED2CB016F3F710519F010F08FEF90E097
:10125000089580E0E3DF8093890181E0DFDF809300
:101260008A0182E0DBDF80938B0183E0D7DF80930C
:101270008C0184E0D3DF80938D0185E0CFDF809304
:101280008E0108951F9381E48EBD84E289BF1FB74C
:10129000F894DFDF1FBF80E01F91089585E091E0A3
:1012A00090931B0180931A0186E191E008950097C5
:1012B00041F0DC01E9E8F1E086E001900D92815017
:1012C000E1F7A1E9B1E0E9E8F1E086E001900D92F3
:1012D0008150E1F788E008958091280190912901DB
:1012E000892B31F0109229011092280181E0089594
:1012F00089E891E061E971E046E050E0E3D10895CA
:1013000082E190E00895A89888EB9BE0FC0131977A
:10131000F1F7A99AFC013197F1F723B3A998019746
:10132000F1F783B3A89A90E08C739070880F991F9F
:10133000880F991F30E02C733070359527953595BF
:101340002795822B8095982F83FD03C040E850E0BD
:1013500002C040E050E091FF02C04FEF50E090FD2E
:1013600003C020E830E002C020E030E092FF02C07D
:101370002FEF30E02093990140939A0110929B0146
:1013800087FF03C081E080939B0196FF05C0809199
:101390009B01826080939B0195FF05C080919B011A
:1013A000846080939B0194FF05C080919B018860BD
:1013B00080939B0108951F931FB7F894B99AC19821
:1013C00084B3837C84BB85B38C6385BB85B3836026
:1013D00085BB84B3836084BB96DF1FBF80E01F9111
:1013E000089589E491E090932F0180932E018AE281
:1013F00091E00895009741F0DC01E9E9F1E083E034
:1014000001900D928150E1F7ACE9B1E0E9E9F1E03A
:1014100083E001900D928150E1F783E0089580917F
:101420003C0190913D01892B31F010923D011092C9
:101430003C0181E0089589E991E06CE971E043E0C5
:1014400050E040D108958FB7F894B99AC198BD9AE9
:10145000C59AA09AA89A94B3917C94BB95B39E63C5
:1014600095BB8FBF80E008958F929F92AF92BF92FD
:10147000CF92DF92EF92FF920F931F93DF93CF9360
:10148000CDB7DEB762970FB6F894DEBF0FBECDBF03
:10149000A8988CE291E00197F1F760E070E0DE013E
:1014A00011961FE060FF04C0C59A999BFECF03C050
:1014B000C5989999FECF43B350E09A0128703070D7
:1014C00035952795CA0180719070F3E095958795C1
:1014D000FA95E1F7282BCA0184709070880F991F44
:1014E000282B4072507035E0559547953A95E1F7B5
:1014F000242BFD01E60FF71F212720836F5F7F4F0D
:101500006231710579F6C59AA89A89818F3009F000
:1015100046C08A818F3009F042C093E0E92EF12C59
:10152000EC0EFD1E26E030E0CC24DD244E010894B4
:10153000811C911C87E0A82EB12CAC0EBD1ED701DA
:101540008C918E3019F08F3021F406C063E070E08A
:1015500005C060E070E002C062E070E08401020F4C
:10156000131FF601E156FE4F40E050E006C0D801DF
:101570008D918D0181934F5F5F4FDA01A20FB31FF1
:1015800046175707A4F30894E11CF11CE3E0F0E0D0
:10159000CE0EDF1EEA14FB0411F09D01D0CF62963F
:1015A0000FB6F894DEBF0FBECDBFCF91DF911F9174
:1015B0000F91FF90EF90DF90CF90BF90AF909F90F2
:1015C0008F9008958BE791E09093430180934201BF
:1015D0008FE292E090934701809346018EE391E081
:1015E00008950F931F93CF93DF938C01662311F41B
:1015F00080E048C083E06802C00111240397EC0139
:10160000C156DE4FDC01A555BE4FFE0183E00190BF
:101610000D928150E1F7888180FD03C0E0E8F0E0A1
:1016200002C0E0E0F0E081FF02C0EFEFF0E082FDF9
:1016300003C040E850E002C040E050E083FF02C039
:101640004FEF50E0898180FD02C020E001C022E020
:1016500081FD246082FD216083FD28608A8180FDF8
:10166000206481FD206282FD206183FD2068D80115
:101670006C9311964C9311971296EC9312971396C4
:101680002C9384E0DF91CF911F910F910895282F23
:101690008091500190915101892B31F010925101AC
:1016A0001092500181E00895215063E02602B001BC
:1016B0001124CB0181569E4F65557E4F43E050E08B
:1016C00001D00895FB01DC0104C08D9101908019C7
:1016D00021F441505040C8F7881B990B0895AA1B6C
:1016E000BB1B51E107C0AA1FBB1FA617B70710F00D
:1016F000A61BB70B881F991F5A95A9F7809590953F
:0A170000BC01CD010895F894FFCF5D
:10170A00FF5A5A3403500050004D0032005500531E
:10171A000042002D00740068006F006D00610073C4
:10172A000070006600650069006600650072002EA0
:10173A00006E006500740009022200010100803277
:10174A00090400000103000000092101010001222F
:10175A0000000705810308000A3403530065006787
:10176A000061004D0075006C00740069007400612E
:10177A000070005F00550053004200010032000073
:10178A000000000000D505A6054D06EC0501000184
:10179A000032000000120000009C070107C307EE98
:1017AA000701000100310000001200000057085F25
:1017BA00087A088008FF01003200000000000000DB
:1017CA00420929096C095709010001003200000089
:1017DA0000000000DB0983090F0AFA09010004006E
:1017EA00B400000012000000230A340A470BF10A71
:0217FA000100EC
:00000001FF
